:1000000079C0000093C0000091C000008FC00000C4
:100010008DC000008BC0000089C0000087C00000B8
:1000200085C0000083C0000081C0000091C30000B3
:100030007DC000007BC0000079C0000077C00000D8
:1000400075C0000073C0000071C000006FC00000E8
:100050006DC000006BC0000069C0000067C00000F8
:1000600065C0000063C0000061C000005FC0000008
:100070005DC000001201100102000008EB034420E3
:1000800000000102DC0109023E00020100C0320949
:1000900004000001020201000524000110042402F2
:1000A000060524060001070582030800FF09040174
:1000B00000020A0000000705040210000007058383
:1000C00002100000040309041803620069007400B0
:1000D000770069007A0061007200640000001C0370
:1000E00043004400430020005500530042004900F3
:1000F0004F00000011241FBECFEFD2E0DEBFCDBF06
:1001000011E0A0E0B1E0EEE7F1E102C005900D9250
:10011000AC33B107D9F711E0ACE3B1E001C01D92F7
:10012000AD38B107E1F746D10C94BD0869CF07C0DF
:10013000EFE4FFE03197F1F700C00000019700976E
:10014000B9F70895982F905D9A3310F4892F01C064
:10015000895C90E06CE371E0A6C71F93182F82952D
:100160008F70F0DF812F8F70EDDF1F9108951F9347
:10017000182F892FF2DF812FF0DF1F9108958091D2
:100180007F01EFE5F1E0E80FF11D80810895909186
:100190007F01EFE5F1E0E90FF11D80819F5F909312
:1001A0007F010895813418F08F7D8753089580531F
:1001B0000895EF92FF920F931F93CF93DF9301C0A7
:1001C000E6DFDDDF8032E1F3C0E0D0E00BC08E017E
:1001D00094E0000F111F9A95E1F7E4DFC82FD0E0FB
:1001E000C02BD12BD4DF803221F08A3011F08D303A
:1001F00071F7CE01DF91CF911F910F91FF90EF909A
:100200000895EF92FF920F931F93CF93DF93BFDF79
:100210008337F9F0843740F4833681F08037A9F1D1
:10022000813609F061C021C0873709F449C08A3797
:1002300009F458C0843709F057C038C0BADF9C01B0
:10024000FC01E85AFE4F10822B5C3E4FF901808181
:100250002BC0AFDF9C01FC01E85AFE4F10822B5CE3
:100260003E4FF90180816ED13FC0A3DFE82EE70148
:100270007E01F92EE7019DDFF701EF5AFE4F8083E3
:10028000C85ADE4F81E088832FC093DFE82FEF014B
:100290007E01F92EE7018DDF8C01CB5CDE4F88817A
:1002A00051D1C80144DF88812FD11EC082DFEC010B
:1002B00080E091E06CE371E022D7CE0158DF14C0FA
:1002C00078DFE82FEF017E01F92E86E156D181E833
:1002D0008093800089E080938100F0928900E09211
:1002E000880002C00C940018DF91CF911F910F91EC
:1002F000FF90EF900895CF92DF92EF92FF920F93CD
:100300001F93CF93DF9338E5E32E31E0F32ECAE459
:10031000D1E005E311E021E5C22E21E0D22EF70164
:1003200081917F01882381F0F60180819881890F76
:10033000888387FF06C080588883F801808102D1B6
:1003400003C0F8018081E0D021960F5F1F4F089411
:10035000C11CD11CFFE5EF16F1E0FF0601F7DF91AC
:10036000CF911F910F91FF90EF90DF90CF90089564
:10037000CF93DF9384B7877F84BF88E10FB6F8946B
:1003800080936000109260000FBE90E080E80FB68E
:10039000F89480936100909361000FBECAD1C5E3C9
:1003A000D1E08991EAD081E0CC33D807D1F7DF9151
:1003B000CF910895FF920F931F93CF93DF93D8DFD0
:1003C0008FE191E06CE371E029D5789482E1D5D09A
:1003D00088E1D3D0FF24C0E0D0E000E010E08091BD
:1003E0002C0180FF12C0FF2091F486E091E06CE3C5
:1003F00071E085D680E191E06CE371E080D68AE11E
:1004000091E06CE371E07BD602C0FF2402C0FF24C0
:10041000F3948FE191E0D5D4BC01181619061CF5B0
:10042000CF31D1052CF08FE191E068E052D514C0B6
:10043000FE01E15AFE4F80838D30910519F08A301C
:10044000910569F410927F018FE591E0DADE8AE18F
:1004500091E06CE371E053D6C0E0D0E004C0219697
:100460008FE191E036D58FE191E023D597D48FE8E5
:1004700091E00197F1F700C000003DDF0F5F1F4FD3
:1004800093E10938190744F082E15CD087E2013139
:1004900018070CF0A2CFA3CF82E136D0A0CF0895E9
:1004A00008958FE191E049C58FE191E08FC59230C9
:1004B00029F0933041F09130E9F417C02EE330E099
:1004C000E6E8F0E01BC0813041F0813018F0823066
:1004D00089F406C0E4ECF0E005C0E8ECF0E002C00E
:1004E000EEEDF0E0249130E009C022E130E0E4E7F5
:1004F000F0E004C020E030E0E0E0F0E0DA01119646
:10050000FC93EE93C9010895982F977021E030E095
:1005100001C0220F9A95EAF7887F803149F088312F
:1005200061F0883071F485B12095282325B90895AC
:1005300088B12095282328B908958BB120952823C8
:100540002BB90895982F977021E030E001C0220F59
:100550009A95EAF7887F803141F0883151F08830F0
:1005600059F485B1282B25B9089588B1282B28B9CD
:1005700008958BB1282B2BB90895982F977021E0FF
:1005800030E001C0220F9A95EAF7887F803141F070
:10059000883151F0883059F484B1282B24B908955A
:1005A00087B1282B27B908958AB1282B2AB9089535
:1005B000382F282F2CC02093E900231721F4762F01
:1005C000942F50E006C07091EC009091ED00509196
:1005D000F00091FF1BC08091EB008E7F8093EB00B9
:1005E0008091ED0082708093ED008091EB0081603E
:1005F0008093EB007093EC009093ED005093F0002B
:100600008091EE0087FD02C080E008952F5F2530C5
:1006100090F23093E90081E008958091850188236C
:100620009CF404C0809184018823B9F08091E80093
:1006300082FFF8CF8091E8008B778093E8000895DF
:1006400080918401882349F08091E80080FFF8CFF1
:100650008091E8008E778093E80008954091E4004F
:100660005091E50024E68091EC0080FF05C0809168
:10067000E80080FF05C022C08091E80082FD1EC016
:1006800080918401882311F482E00895853011F46B
:1006900083E008958091EB0085FF02C081E008951A
:1006A0008091E4009091E50084179507E1F2222300
:1006B00011F484E008952150AC01D5CF80E0089575
:1006C00041D043D08091D800982F9F779093D80045
:1006D00080688093D8008091D8008F7D8093D80067
:1006E00084E089BD89B5826089BD09B400FEFDCF73
:1006F0001092840110928201109281011092800167
:1007000080E060E042E054DF8091E1008E7F8093E2
:10071000E1008091E20081608093E2008091E2003C
:1007200088608093E2008091E0008E7F8093E000FB
:100730000895E3E6F0E080818E7F808381E08093FE
:100740008301BECF1092E20008951092E100089557
:100750001F920F920FB60F9211242F933F934F9336
:100760005F936F937F938F939F93AF93BF93EF9319
:10077000FF938091E10082FF0AC08091E20082FF36
:1007800006C08091E1008B7F8093E10008D28091C8
:10079000E10080FF17C08091E20080FF13C08091CC
:1007A000E2008E7F8093E2008091E200806180937E
:1007B000E2008091D80080628093D80019BC10922A
:1007C00084016EDE8091E10084FF2EC08091E20002
:1007D00084FF2AC084E089BD89B5826089BD09B4DF
:1007E00000FEFDCF8091D8008F7D8093D80080914E
:1007F000E1008F7E8093E1008091E2008F7E809304
:10080000E2008091E20081608093E20080918201A9
:10081000882331F48091E30087FD02C081E001C0AC
:1008200084E0809384013BDE8091E10083FF22C05D
:100830008091E20083FF1EC08091E100877F80935A
:10084000E10082E080938401109282018091E100B6
:100850008E7F8093E1008091E2008E7F8093E200A2
:100860008091E20080618093E20080E060E042E0FD
:100870009FDE95D1FF91EF91BF91AF919F918F91A5
:100880007F916F915F914F913F912F910F900FBE8C
:100890000F901F9018950F931F93DF93CF93CDB7B1
:1008A000DEB7AC970FB6F894DEBF0FBECDBF809118
:1008B000F100809385018091F10080938601809101
:1008C000F1009091F100E7E8F1E0809387019093C7
:1008D00088018091F1009091F100809389019383C8
:1008E0008091F1009091F10080938B019583DCDD84
:1008F0008091E80083FF3AC18091850130918601A3
:10090000353009F487C0363040F43130C9F1313028
:1009100070F0333009F02AC133C0383009F4F8C020
:10092000393009F407C1363009F020C199C0803848
:1009300021F0823809F01AC108C09091800180919D
:100940008101882399F0926011C08091890187709C
:100950008093E9008091EB0090E025E096958795E3
:100960002A95E1F7982F91701092E9008091E800A4
:10097000877F8093E8009093F1001092F100D3C03C
:10098000882319F0823009F0F1C090E08F719070E7
:10099000009721F0029709F0E9C00CC0809187010F
:1009A000813009F0E3C010928101333069F5809302
:1009B00081012AC080918701882331F52091890126
:1009C000277009F4D3C02093E9008091EB0080FFE9
:1009D0001BC0333021F48091EB00806213C0809102
:1009E000EB0080618093EB0081E090E002C0880F13
:1009F000991F2A95E2F78093EA001092EA0080910D
:100A0000EB0088608093EB001092E9008091E80091
:100A1000877F8CC0882309F0A9C0109187011F77B8
:100A20000FB7F8948091E800877F8093E800F5DDA8
:100A30008091E80080FFFCCF8091E3008078812BDB
:100A40008093E3008091E30080688093E3001123AA
:100A500011F482E001C083E0809384010FBF86C05F
:100A60008058823008F082C080918701909188017F
:100A700023E08C3D920709F033C083E08C838AE247
:100A80008B837FB7F894DE0115966EE040E050E06E
:100A900011E2E62FF0E010935700849140FF03C06D
:100AA00082958F706F5F8F70282F30E08A3018F03A
:100AB000C901C79602C0C901C0968D939D934F5F2F
:100AC0005F4F4431510529F77FBF8091E800877F50
:100AD0008093E800CE0103966AE270E061D012C014
:100AE00060918901AE014F5F5F4FE1DCBC0100976F
:100AF00009F43CC08091E800877F8093E8008981F9
:100B00009A81EBD08091E8008B778093E8002EC02B
:100B1000803861F58091E800877F8093E8008091BC
:100B200082018093F1008091E8008E778093E80045
:100B300074DD1CC08823D1F4909187019230B0F409
:100B40008091E800877F8093E8009093820165DDC3
:100B500080918201882331F48091E30087FD02C0F7
:100B600081E001C084E0809384019BDC8091E800F7
:100B700083FF0AC08091EB0080628093EB0080913C
:100B8000E800877F8093E800AC960FB6F894DEBF4C
:100B90000FBECDBFCF91DF911F910F9108950895A2
:100BA0009C0140918B0150918C014617570718F416
:100BB000F90190E03DC06115710511F0AB01F8CF6E
:100BC0008091E8008E778093E80040E050E0F0CF1D
:100BD000809184018823F1F18530F1F18091E80062
:100BE00083FF02C081E008958091E80082FD2CC05F
:100BF0008091E80080FF1CC08091F200282F30E037
:100C000007C081918093F100415050402F5F3F4FCA
:100C10004115510519F02830310598F390E028303E
:100C2000310509F491E08091E8008E778093E80027
:100C30004115510569F6992359F606C08091840142
:100C4000882341F0853041F08091E80082FFF6CFA3
:100C500080E0089582E0089583E008959C01611585
:100C6000710529F48091E8008B778093E800F90101
:100C700020C080918401882361F1853061F18091E9
:100C8000E80083FF02C081E008958091E80082FFC0
:100C9000F0CF06C08091F10081936150704021F047
:100CA0008091F2008823B1F78091E8008B778093E0
:100CB000E80061157105E9F606C08091840188237A
:100CC00041F0853041F08091E80080FFF6CF80E070
:100CD000089582E0089583E008959C0140918B017E
:100CE00050918C014617570718F4F90190E040C065
:100CF0006115710511F0AB01F8CF8091E8008E7796
:100D00008093E80040E050E0F0CF80918401882398
:100D100009F440C0853009F43FC08091E80083FFAA
:100D200002C081E008958091E80082FD2DC080918D
:100D3000E80080FF1DC08091F200282F30E008C03D
:100D400084918093F1003196415050402F5F3F4F86
:100D50004115510519F02830310590F390E0283005
:100D6000310509F491E08091E8008E778093E800E6
:100D70004115510551F6992341F606C08091840131
:100D8000882341F0853041F08091E80082FFF6CF62
:100D900080E0089582E0089583E008951F93809194
:100DA0008401882361F01091E9001092E90080919C
:100DB000E80083FF01C06FDD17701093E9001F91F9
:100DC0000895FC0180918401843021F58785908904
:100DD000A189B2890097A105B105E1F085818093D1
:100DE000E9008091E80082FF15C08091F20088231D
:100DF00019F42FEF3FEF04C08091F100282F30E06D
:100E00008091F200882341F48091E8008B778093F1
:100E1000E80002C02FEF3FEFC9010895FB012EE06B
:100E2000DB011D922A95E9F723E023832EE837E0C2
:100E30003187208721E237E03387228795878487AF
:100E40000895FC0184859585BCDF9C0197FF02C055
:100E50002EEF3FEFC90108950895FC0180918401B0
:100E6000843011F587859089A189B2890097A10501
:100E7000B105D1F081818093E9008091F20088234F
:100E8000A9F09091E8008091E8008E778093E800C7
:100E900095FD0CC0E3DB982F882349F48091E8008E
:100EA0008E778093E80003C092E001C090E0892F24
:100EB0000895FC0180918401843051F487859089E4
:100EC000A189B2890097A105B10511F0CF01C5CF65
:100ED00008951F93FC01162F809184018430D9F46A
:100EE00087859089A189B2890097A105B10599F0FC
:100EF00081818093E9008091E80085FD08C08091A0
:100F0000E8008E778093E800A9DB882329F410930A
:100F1000F10080E001C082E01F910895282FFB01BD
:100F200084859585622FD5DF882319F420E030E091
:100F300002C02FEF3FEFC90108951F93CF93DF93B6
:100F4000EC010D96FC0189E0DF011D928A95E9F71D
:100F500011E08981181729F4EA81FB818C8162E014
:100F600010C08D81181731F4EE81FF81888562E011
:100F700030E008C08985181709F5EA85FB858C855E
:100F800063E031E0882311F440E001C044E020E058
:100F900088E090E003C02F5F880F991F8E179F078E
:100FA000D0F36295660F660F607C632B42602295DA
:100FB000207F422B812FFCDA882321F01F5F153020
:100FC00041F681E0DF91CF911F910895CF93DF9398
:100FD000EC018091E80083FF63C0888190E020915C
:100FE000890130918A012817390709F059C0809189
:100FF0008601813261F0823220F4803209F050C0E3
:101000001BC0823279F1833209F04AC03BC0809123
:101010008501813A09F044C08091E800877F809380
:10102000E800CE010F9667E070E0BADD8091E8003D
:101030008B778093E80034C080918501813281F5FF
:101040008091E800877F8093E800CE010F9667E0EB
:1010500070E004DE8091E8008E778093E800CE0196
:10106000FBDE1EC0809185018132D1F48091E800C1
:10107000877F8093E800D1DA809187018D87CE0148
:10108000EBDE0EC080918501813251F48091E80041
:10109000877F8093E800C1DACE0160918701DCDEB2
:1010A000DF91CF9108950F931F93CF93DF938C011E
:1010B000EB018B8181FF1BC082FF0DC02E813F8120
:1010C0008C819D812817390764F4E881F9810193A7
:1010D000F983E88306C0E885F985802F0995009794
:1010E00031F48E819F8101969F838E8302C00FEF22
:1010F0001FEFC801DF91CF911F910F910895EF92DB
:10110000FF920F931F93CF93DF937C01EB018B81B1
:1011100081FF11C000E010E008C0E885F985BE013C
:101120000995009711F00FEF1FEFF70181917F01F3
:10113000882399F702C00FEF1FEFC801CDB7DEB7C4
:10114000E6E00CC02A88398848885F846E847D84F4
:101150008C849B84AA84B984C884DF80EE80FD805F
:101160000C811B81AA81B981CE0FD11D0FB6F894D5
:0E117000DEBF0FBECDBFED010895F894FFCF96
:10117E00676F743A200043444320757362696F00B1
:10118E0020686464706F776572000D0A3E2000005F
:10119E000310000004100000020800000000000010
:0C11AE00000000000018191A1B1C1D1E78
:00000001FF
